:0200000270008C
:10800000489A0020398507006185070063850700CD
:108010006585070067850700698507000000000087
:108020000000000000000000000000006B85070059
:108030006D850700000000006F850700718507004F
:108040007385070073850700738507007385070034
:108050007385070073850700738507007385070024
:108060007385070073850700738507007385070014
:1080700073850700A9C30700738507007385070090
:1080800073850700BDC70700738507007385070068
:1080900069C407007385070061C107007385070085
:1080A00073850700738507007385070073850700D4
:1080B00073850700738507000000000000000000C2
:1080C00073850700738507007385070073850700B4
:1080D00073850700738507007385070000000000A3
:1080E0000000000000000000000000000000000090
:1080F0000000000000000000000000000000000080
:10810000000000000000000000000000000000006F
:10811000000000000000000000000000000000005F
:1084000010B5054C237833B9044B13B10448AFF3CE
:1084100000800123237010BD5047002000000000A1
:10842000D4CF070008B5034B1BB103490348AFF392
:10843000008008BD0000000054470020D4CF070092
:10844000154B002B08BF134B9D46A3F5803A002126
:108450008B460F461348144A121A00F063F80F4B6C
:10846000002B00D098470E4B002B00D098470020DF
:10847000002104000D000D48002802D00C48AFF385
:10848000008000F02BF82000290004F0F5F900F03E
:1084900011F800BF00000800489A0020000000000A
:1084A00000000000504700205C5400200000000045
:1084B0000000000008B5074B044613B10021AFF3DC
:1084C0000080054B1868836A03B19847204600F086
:1084D00031F800BF0000000068CC070070B50D4DFA
:1084E0000D4C641BA4100026A64209D10B4D0C4C68
:1084F00004F0AEFB641BA4100026A64205D170BD9B
:1085000055F8043B98470136EEE755F8043B984789
:108510000136F2E730470020304700203047002086
:108520003447002002440346934200D1704703F8C9
:10853000011BF9E7FEE700BF0649074A074B9B1AF4
:1085400003DD043BC858D050FBDC03F017FEFFF7F7
:1085500077FF0000E0CF0700C8460020504700200A
:10856000FEE7FEE7FEE7FEE7FEE7FEE7FEE7FEE7E3
:10857000FEE7FEE7204B21491A682F2300BF00BF0A
:1085800000BF00BF00BF00BF00BF00BF8A422FD0A6
:1085900000BF00BF00BF00BF00BF00BF00BF00BFE3
:1085A00000BF00BF00BF00BF00BF00BF00BF00BFD3
:1085B00000BF00BF00BF00BF00BF00BF00BF00BFC3
:1085C00000BF00BF00BF00BF00BF00BF00BF00BFB3
:1085D00000BF00BF00BF00BF00BF00BF00BF00BFA3
:1085E00000BF00BF00BF00BF00BF00BF00BF00BF93
:1085F000013BC3D1704700BF284700200024F4008E
:1086000070B5EFF3108672B60D4A94680123A4B9D1
:1086100093600C4B0C4DD3F8801029401160C3F8C7
:108620008050D3F8841051604FF0FF32C3F884209B
:10863000047006B962B6002070BD0370F9E700BF90
:108640001C50002000E100E0FC06FFBC2DE9F04FCB
:10865000C9B008AA01F1400514464B780E781B04F6
:1086600043EA0663CE7833438E78043143EA062327
:108670008D4244F8043BF0D11024916B16464FEA2A
:10868000F14383EA714383EA9123716A366852F8B1
:10869000045F31440B444FEAB54181EAF51181EAA8
:1086A000D50101340B44402CD363E6D1D0E914E367
:1086B0000093836D0193C36D0293036E0393436E26
:1086C0000493836E0593C36E0693DDE9057BDDE9B4
:1086D000031CDDE901592B4B009E079374464FF0B4
:1086E0000008079B53F8042B07934FEAF12383EA12
:1086F000B11383EA716A08AB53F828301A440AEBC5
:10870000020327EA010A01EA0C028AEA02021A4479
:108710004FEA743A86EA05035A448AEAB40A06EA3A
:10872000050B234083EA0B038AEAB45A08F10108D7
:108730009A44B8F1400F02EB0903BB465244A946E4
:1087400019D172440265009A22444265019A32446A
:108750008265029A2A44C265039A1A44049B0266FF
:108760000B444366059B63448366069B3B44C36698
:1087700049B0BDE8F08F674635468C462646194617
:108780001446AEE794CE07002DE9F04F93B0CDE943
:10879000002002A892F90020B1E8005E06B4AAFB0E
:1087A00009124FF00003EBFB69234FF00004ECFBD0
:1087B00069344FF00005EEFB69454FF00006EBFB16
:1087C0006A63ECFB6A344918524176415B41A9FB6C
:1087D00009784FF0000949F1000918EB0108A0E8F9
:1087E0008001AAFB0A78574158EB0608A0E88001EF
:1087F000EEFB6A454FF0000A4AF1000A4FF0000113
:10880000ECFB6B14EEFB6B454FF00002EEFB6C25AE
:108810005FEA59094941644152416D4149F10009FA
:10882000EBFB6B3A1AEB010AA0E80804ACFB0C6AFC
:1088300066415AEB020AA0E84004AEFB0E6A6E41A4
:108840005AEB090AA0E8400406BC052A00F0E680BD
:10885000A0F11400A1F11401B1E8E043A5FB0E342E
:108860004FF00005E6FB6E454FF00006E7FB6E5645
:108870004FF00007E8FB6E674FF00008E9FB6E78E9
:108880004FF00009DB1864416D4176417F4158EBA0
:10889000080859F1000950F804CB13EB0C0350F809
:1088A00004CB54EB0C0450F804CB55EB0C0550F8FA
:1088B00004CB56EB0C0650F804CB57EB0C0758F1E1
:1088C000000859F10009A0F11400EEFB0E89A0E8A0
:1088D000F803062A00F0A280A0F11800A1F1180107
:1088E000B1E8E047A5FB0E344FF00005E6FB6E450E
:1088F0004FF00006E7FB6E564FF00007E8FB6E678F
:108900004FF00008E9FB6E784FF00009EAFB6E8932
:108910004FF0000ADB1864416D4176417F4158EB0E
:10892000080859EB09095AF1000A50F804CB13EB77
:108930000C0350F804CB54EB0C0450F804CB55EB6B
:108940000C0550F804CB56EB0C0650F804CB57EB53
:108950000C0750F804CB58EB0C0859F100095AF1F8
:10896000000AA0F11800EEFB0E9AA0E8F807072A0B
:1089700054D0A0F11C00A1F11C01B1E8E04FA5FB0F
:108980000E344FF00005E6FB6E454FF00006E7FBA6
:108990006E564FF00007E8FB6E674FF00008E9FBEA
:1089A0006E784FF00009EAFB6E894FF0000AEBFB8E
:1089B0006E9A4FF0000BDB1864416D4176417F41A8
:1089C00058EB080859EB09095AEB0A0A5BF1000B4E
:1089D00050F804CB13EB0C0350F804CB54EB0C040D
:1089E00050F804CB55EB0C0550F804CB56EB0C06B5
:1089F00050F804CB57EB0C0750F804CB58EB0C089D
:108A000050F804CB59EB0C095AF1000A5BF1000B4A
:108A1000A0F11C00EEFB0EABA0E8F80F009B019844
:108A2000D3F8AC3002A9984713B0BDE8F08F00EB43
:108A300081010023884200D3704751F8042D43EA96
:108A400052030B60D307F5E710B5013A52B2130693
:108A500001D5002010BD50F8224051F822309C4230
:108A600005D802F1FF32F2D24FF0FF30F2E70120D9
:108A7000F0E710B500235CB2A24200DC10BD51F853
:108A8000234040F823400133F5E7013910B549B2DE
:108A9000041D0A06CBB204D4013954F82120002A5F
:108AA000F7D001335BB273B103F18042013A50F861
:108AB0002220002022B9013B00EB431318B210BD65
:108AC00052080130F6E71846F9E74A11012350F839
:108AD000220001F01F0103FA01F10840704710B5B0
:108AE00000231A465CB2A14203DCB2FA82F04009CC
:108AF00010BD50F8234001332243F3E7002310B5A3
:108B00001C465AB2914200DC10BD40F823400133AC
:108B1000F7E72DE9F04FA5B01D4604ABCDE90231D2
:108B20008146294610461746FFF7AFFFC0EB851078
:108B300004B2002C2646B8BF04F11F06634246F378
:108B4000471603F01F0304F01F0814A858BFC3F111
:108B500000083146FFF7D2FFB8F1000F30B22DDD2B
:108B600014AB002203EB8000C8F1200C13469D4299
:108B700019D82FB27B00019314AB03EB870705F1E3
:108B8000FF3824AB012603EB8808002C54DA24AB11
:108B900003EB86062A4656F8881C4846FFF769FF0D
:108BA00025B0BDE8F08F57F8236006FA08F10A43B4
:108BB00040F8042B013326FA0CF2D8E714AB2A460E
:108BC000394603EB8000FFF754FFD2E70FFA82FE2D
:108BD0005AF8883C53F82EB024AB03EB82020130E4
:108BE00052F8403C0B44BBEB030334BF012200228C
:108BF0009B4518BF11465CF8882C42F82E30019B2B
:108C000042B29A42E2DB731A5E42294614A85E41E0
:108C1000FFF70DFF24AB03EB8503294653F8402CE7
:108C200058F8403C384643EAC273013C48F8403C9F
:108C300024B2FFF7FCFEA8E724AB0020C6F1010C2C
:108C4000014603EB860A03EB8C0CD8E72DE9F04FC5
:108C500008B4F8CA04B451F8042BA3FB028940F805
:108C6000048B4FF0000AE4FB629A4FF0000BE5FB27
:108C700062AB4FF0000CE6FB62BC4FF0000EE7FB6E
:108C800062CE51F8042B4FF00008E3FB628940F8F4
:108C9000048BE4FB629AE5FB62ABE6FB62BCE7FB9C
:108CA00062CE51F8042B4FF00008E3FB628940F8D4
:108CB000048BE4FB629AE5FB62ABE6FB62BCE7FB7C
:108CC00062CE51F8042B4FF00008E3FB628940F8B4
:108CD000048BE4FB629AE5FB62ABE6FB62BCE7FB5C
:108CE00062CE51F8042B4FF00008E3FB628940F894
:108CF000048BE4FB629AE5FB62ABE6FB62BCE7FB3C
:108D000062CE40F8049B40F804AB40F804BB40F846
:108D100004CB40F804EB0CBC052B00F01E810C6862
:108D2000A0F11400A1F11401A2F1140252F804EB15
:108D30004FF0000550F8046BE4FB6E5652F804EB5C
:108D400050F8047BE4FB6E6752F804EB50F8048B98
:108D5000E4FB6E7852F804EB50F8049BE4FB6E8958
:108D600052F804EB50F804ABE4FB6E9AA0F1140047
:108D700052F8044B51F804EB4FF0000CE4FB6EC5C5
:108D800040F804CB51F804EBE4FB6E5640F8045B6A
:108D900051F804EBE4FB6E6740F8046B51F804EB08
:108DA000E4FB6E7840F8047B51F804EBE4FB6E8939
:108DB00040F8048B51F804EBE4FB6E9AA0E800063F
:108DC000062B00F0CA800C68A0F11800A1F1180170
:108DD000A2F1180252F804EB4FF0000550F8046BB2
:108DE000E4FB6E5652F804EB50F8047BE4FB6E672C
:108DF00052F804EB50F8048BE4FB6E7852F804EB65
:108E000050F8049BE4FB6E8952F804EB50F804AB75
:108E1000E4FB6E9A52F804EB50F804BBE4FB6EAB33
:108E2000A0F1180052F8044B51F804EB4FF0000C7D
:108E3000E4FB6EC540F804CB51F804EBE4FB6E563E
:108E400040F8045B51F804EBE4FB6E6740F8046BF8
:108E500051F804EBE4FB6E7840F8047B51F804EB26
:108E6000E4FB6E8940F8048B51F804EBE4FB6E9A46
:108E700040F8049B51F804EBE4FB6EABA0E8000C57
:108E8000072B6AD008B40C68A0F11C00A1F11C01EA
:108E9000A2F11C0252F804EB4FF0000550F8046BED
:108EA000E4FB6E5652F804EB50F8047BE4FB6E676B
:108EB00052F804EB50F8048BE4FB6E7852F804EBA4
:108EC00050F8049BE4FB6E8952F804EB50F804ABB5
:108ED000E4FB6E9A52F804EB50F804BBE4FB6EAB73
:108EE00052F804EB50F804CBE4FB6EBCA0F11C007C
:108EF00052F8044B51F804EB4FF00003E4FB6E35DD
:108F000040F8043B51F804EBE4FB6E5640F8045B78
:108F100051F804EBE4FB6E6740F8046B51F804EB86
:108F2000E4FB6E7840F8047B51F804EBE4FB6E89B7
:108F300040F8048B51F804EBE4FB6E9A40F8049B74
:108F400051F804EBE4FB6EAB40F804AB51F804EBD2
:108F5000E4FB6EBCA0E8001808BCBDE8F08F30B59B
:108F60001C4691B0054693F900306846FFF76EFE47
:108F7000D4F8AC3069462846984711B030BDF0B5FA
:108F8000154689B01C4607460E461A4629466846CD
:108F9000FFF7FAFB23466A4639463846FFF7DFFFFC
:108FA00023462A4669466846FFF7D9FF23466A46A4
:108FB00031463046FFF7D3FF09B0F0BD0000000096
:108FC000C3F10803DB0070B50133002403A500BF23
:108FD0005B1920C940CAAD1B20C0184720C940CA30
:108FE000B54120C020C940CAB54120C020C940CAEF
:108FF000B54120C020C940CAB54120C020C940CADF
:10900000B54120C020C940CAB54120C020C940CACE
:10901000B54120C06441B4FA84F0400970BD00BF7E
:10902000C3F10803DB0070B50133002403A500BFC2
:109030005B1920C940CAAD1920C0184720C940CAD1
:10904000754120C020C940CA754120C020C940CA0E
:10905000754120C020C940CA754120C020C940CAFE
:10906000754120C020C940CA754120C020C940CAEE
:10907000754120C06441204670BD00BFF0B5082294
:1090800089B00C460646FFF7F4FCCB6A03930B6BE2
:1090900004934B6B05938B6B0693CB6B0793002765
:1090A00008236A4669466846CDE901770097FFF7CD
:1090B000B7FF082305466A4631463046FFF7B0FF42
:1090C000236B0393636B0493A36B0593E36B0544DA
:1090D000CDE906376A46082369466846FFF7A0FFD0
:1090E000082305446A4631463046FFF799FF236A54
:1090F0000093636A0193A36A0293A36B0693E36BE5
:109100000793054408236A4631463046CDE9047783
:109110000397FFF785FF636A0093A36AA26B01932D
:10912000E36A02930492636BE26B0393CDE9052338
:10913000236A0793054408236A4631463046FFF701
:109140006FFFE36A0093236B0193636B0293236ABF
:109150000693A36A0793054408236A4631463046BE
:10916000CDE904770397FFF72BFF236B0093636B25
:109170000193A36B0293E36B0393636A0693E36A21
:1091800007932D1A08236A4631463046CDE9047705
:10919000FFF716FF636B0093A36B0193E36B0293DE
:1091A000236A0393636A0493A36ACDE90537236BAB
:1091B00007932D1A08236A4631463046FFF700FF11
:1091C000A36B0093E36BCDE90137636A0393A36A52
:1091D0000493E36ACDE90537636B07932D1A0823DF
:1091E0006A4631463046FFF7EBFE2D1A0D4C0FD480
:1091F00035B9082231462046FFF726FC01280FD05A
:109200000823224631463046FFF7DAFE2D1AEFE7F3
:109210000823224631463046FFF702FF2D18F7D4C7
:1092200009B0F0BDACCC070070B5036813F00105C0
:109230000646144605D013460A460146FFF7F0FEDF
:10924000054621463046FFF7F2FB45B104F1804266
:10925000013A56F8223043F0004346F8223070BD00
:10926000F0B50F46A1B006461946384615461C46CD
:10927000FFF735FC20B13046FFF740FC21B0F0BDD0
:10928000224639466846FFF7F4FB294608A8FFF74F
:10929000F0FB10A82146FFF731FC012318A810931A
:1092A000FFF72CFC224608A96846FFF7CDFB28B93A
:1092B000224610A93046FFF7DCFBDFE7009BDA0708
:1092C00009D421466846FFF7B2FB2246294610A87A
:1092D000FFF7AAFFE6E7089BDB0707D4214608A8AB
:1092E000FFF7A5FB2246294618A8F1E700282346E8
:1092F0001CDD08AA69466846FFF762FE21466846FB
:10930000FFF795FB224618A910A8FFF79DFB002840
:1093100005DA10A923462A460846FFF781FE10A960
:10932000234618AA0846FFF74BFECEE708A96A466F
:109330000846FFF745FE214608A8FFF778FB2246BE
:1093400010A918A8FFF780FB002805DA18A9234602
:109350002A460846FFF764FE18A9234610AA0846C5
:10936000FFF72EFEBEE770B59DF910401E4623465E
:109370000546FFF725FE38B12346324629462846E2
:10938000BDE87040FFF74CBE70BD2DE9F0438BB0D7
:109390001446129D15F9046B00961F4680468946B7
:1093A0002B460246214602A8FFF7DDFF02A9129ACA
:1093B0000846FFF7E9F9129B02AA41464046FFF72B
:1093C000CEFD129B02AA21462046FFF7C8FD2B4680
:1093D0004A46394638460096FFF7C5FF129A394685
:1093E00002A8FFF7D1F902A92B464246084600968B
:1093F000FFF7B9FF02A92B46224608460096FFF761
:10940000B2FF2B464246214620460096FFF7ABFFAF
:10941000129B224649464846FFF7A1FD2B4602AA69
:10942000414620460096FFF79EFF129B2246394692
:109430003846FFF794FD2B464A4639463846009693
:10944000FFF791FF324602A92046FFF712FB0BB04F
:10945000BDE8F0832DE9F04FEBB09346749F059182
:10946000B7F9022097F9004012F11F0148BF02F13D
:109470003E0141F347120292013A4FEA82096AA97A
:1094800012AE82460DF1280801EB0900002140F8D8
:10949000C01C46F8221048F8221097F901103046F7
:1094A0000D460A46002A40F0268103EB4103002DB9
:1094B00040F0278121463046FFF711FB002840F09D
:1094C00016814046FFF70BFB0490002840F00F8107
:1094D00007F12403029A039331461846FFF7B4FAC2
:1094E000012840F00481029A03984146FFF7ACFA44
:1094F000012840F0FC8042AEDDE902323046FFF741
:10950000AFFE6AAB9944B7F9023049F8605C13F1D9
:109510001F0548BF03F13E05DA1D48BF03F10E02E7
:109520006D11D2100DF5A4784FFA85F9934549468F
:10953000404628BF9346FFF7E1FA059B08EB0B0274
:109540005B4405998B4240F0E280B7F902304FEA64
:10955000CB0B9B4515D9ABEB030B08EB8505002224
:10956000CBF12000A845C0F0D7804A464146039879
:10957000FFF76AFA012804D04B46039A4046FFF7EA
:109580001FFD5AAD2846029B324652A9FFF75EFBEB
:10959000DDE90232294652A8FFF7BBFA2846029BB2
:1095A000324612A9FFF752FB4FEA840BDDE9023283
:1095B00029464AA8FFF7ADFA05EB0B0922465146AA
:1095C0002846FFF756FA07F144080AEB0B01484614
:1095D000FFF74FFA41462AA8FFF74BFA08EB0B01B9
:1095E00022A8FFF746FA3B1D29462AAA30460094D6
:1095F0000593FFF7B8FE4B462A4622A92AA80097F2
:10960000FFF7C3FE23463A1D31463046FFF728FEDA
:109610003246494628463B46FFF7B1FC00230299F3
:1096200052A8CDE90638CDE908A5FFF72EFA029930
:1096300080464AA8FFF729FA8045B8BF80461FFA3E
:1096400088F808F1FF352DB2294652A8FFF73DFAF8
:10965000294610F1000A4AA818BF4FF0010AFFF787
:1096600034FA002814BF022300234AEA030A0DF14A
:109670001809224659F82A500DF1E80929464846AA
:109680000DF1C80AFFF7F5F905EB0B015046FFF79E
:10969000F0F921463046FFF731FA01234293A8F151
:1096A00002080FFA88F8B8F1000F3EDA2346059A4F
:1096B00031463046FFF7D4FD3B46324651464846D8
:1096C000FFF75DFC029A03984946FFF7BDF90128B0
:1096D00004D0DDE902324846FFF772FC013C64B277
:1096E00012AA230663D5049BB3FA83F56D092846B5
:1096F0006BB0BDE8F08F013A13F802C002F800C069
:10970000D0E6013D13F8012D08F80520CFE613F847
:10971000011D02F8011D14E755F8041D21FA0BF391
:1097200013432B6001FA00F21CE73B463246D7F8A0
:10973000A45051464846A847414652A8FFF7C5F9EC
:109740004146051C4AA818BF0125FFF7BEF90028AD
:1097500014BF022300231D4306AB53F825501DB34D
:10976000224629462AA8FFF784F905EB0B0122A817
:10977000FFF77FF93B46324622A92AA8FFF7FFFBF5
:10978000059B00942AAA49461AA8FFF7ECFD534608
:109790004A4622A92AA80097FFF7F7FD3B461AAAD6
:1097A00031463046FFF7DBFB08F1FF3879E752F826
:1097B000241059F824304B40049919430491013C7A
:1097C0008FE770B59DF910401E4623460546FFF70A
:1097D00027FC30B9224629463046FFF735F90128E3
:1097E00007D02346324629462846BDE87040FFF799
:1097F000E7BB70BD2DE9F04115468AB004468846A6
:109800001C22002103A8FEF78DFE2E1D95F9007085
:1098100003232A46414620460293FEF7B5FF33460E
:1098200002AA214620460097FFF79DFD2B4642469F
:1098300021462046FFF793FB0097334605F184024B
:1098400021462046FFF7BDFF0AB0BDE8F0812DE9B3
:10985000F04793F9006092B00446894610463146BD
:1098600015469846FFF73BF9002840F091804246A4
:1098700049460AA8FEF788FF43460AAA214602A8DD
:10988000FFF76DFB0AA908464246FEF77DFF4346F7
:109890002A4649464846FFF762FB08F1040742465C
:1098A00029462846FEF770FF3B462A4621462046B9
:1098B0000096FFF786FF3B462A4629462846009633
:1098C000FFF77FFF3B462A46214628460096FFF7D2
:1098D0004AFD43462A4621462046FFF740FB3B46C9
:1098E0002246214628460096FFF76BFF3B4600962E
:1098F0002A4621462046FFF764FF2368DB074AD546
:1099000033463A4621462046FFF78AFB31468246D7
:109910002046FFF78CF806F18043013B54F8230002
:1099200040EACA7044F82300424621462846FEF722
:109930002BFF3B4602AA294628460096FFF713FD57
:109940003B4602AA294628460096FFF70CFD02A9CD
:1099500008463B462A460096FFF705FD434602AA05
:1099600021462046FFF7FBFA0AAA3B46104621464D
:109970000096FFF7F8FC324629462046FFF779F8B3
:1099800049462846FFF775F80AA94846FFF771F8D7
:1099900012B0BDE8F08731462046FFF748F8C3E72C
:1099A00010B5012203680446984710B1A368013B33
:1099B000A36010BD10B50B689A684B680024C0E91D
:1099C0000243C0E9002294782344036192F90340E2
:1099D000234443614B68036101F10C0343615378F5
:1099E00003F0C003802B04BF0431016110BD436844
:1099F0001A44426011B101399A4201D101207047E5
:109A000013F8010B01F8010FF6E72DE9F3470025E4
:109A100080460F462E462C46D8F8083023B30DF169
:109A200007014046FFF7BCFFF0B19DF807C00CF0FE
:109A30007F025FFA82F9A4F12003C4F1200109FA40
:109A400003F329FA01F109FA04F20B431CF0800F29
:109A500045EA020546EA030604F1070402D1C7E914
:109A6000005602E0462CD7D1002002B0BDE8F087B6
:109A7000F7B50F4669461646FFF7C7FFB0B1DDE9F7
:109A80000013002501F001044A0842EAC37254EAB7
:109A900005014FEA530314BFDD431D463B7914BF54
:109AA000D4431446082B03D1C6E9004503B0F0BDEA
:109AB000042B08D134602246D317AB4206BFA24222
:109AC00001200020F2E7022B03D123B233801AB227
:109AD000F2E7012B03D163B233705AB2ECE70020F6
:109AE000E4E773B50C4669461646FFF78EFF68B18A
:109AF0002379082B0CD1DDE90045C6E90045DDE9F5
:109B00000023AB4206BFA2420120002002B070BD7C
:109B1000042B04D1009B33601C460025EFE7022B89
:109B20004FF0000004D1009B33809CB20546E6E76D
:109B3000012BEBD1009B337003F0FF04F6E737B540
:109B40000D4669461446FFF760FF30B12A79082AAE
:109B5000DDE9003103D1C4E9003103B030BD042A8E
:109B600018464FEAE37108D123601A460B468B4230
:109B700006BF824201200020EFE7022A04D11BB277
:109B800023801AB2D317F2E7012A03D15BB2237004
:109B90005AB2F7E70020E0E72DE9F3418368074672
:109BA000884623B90026304602B0BDE8F0810DF1A9
:109BB0000701FFF7F5FE06460028F3D09DF80740A1
:109BC000220616D504F07F040725BB68002BE9D0D8
:109BD0000DF107013846FFF7E3FE0028E2D09DF8BB
:109BE000072002F07F03AB401C43130605F1070575
:109BF00002D4C8F80040D6E7232DE6D1D2E773B5EA
:109C00000D4601A90446FFF7C7FF064618B900260E
:109C1000304602B070BD94E80F0085E80F0001994E
:109C20008A42F4D3A960A3685B1AA360F0E700003E
:109C300030B5044685B01546A9B90268114B9A4261
:109C400011D0102D06D82A4669462046FFF7F0FFAE
:109C500005B030BD102269462046FFF7E9FF002815
:109C6000F6D0103DEDE7A368AB4201D20020EFE74C
:109C700023682A46204698470028F7D0A3685D1B32
:109C8000A560E5E7EF990700F7B50E4601A907467D
:109C90001546FFF781FFA8B1019A0123D3184FF0B1
:109CA000000404D2717801F0C001802901D120465E
:109CB00008E031799942FAD329463846FFF7B8FFD0
:109CC000019BEC5403B0F0BD73B50D4601A90646E7
:109CD0001446FFF761FF90B1019AFF2A11D86B7803
:109CE00003F0C003802B02F101010AD02B798B42D3
:109CF00007D32146304601F8012BFFF799FF02B048
:109D000070BD0020FBE713B5144669460822FFF733
:109D10008FFF18B1DDE90023C4E9002302B010BDB4
:109D200013B5144604220DEB0201FFF781FF08B1C1
:109D3000019B236002B010BD13B5044605291FD84E
:109D4000DFE801F0030F151E1E1C012201A92046A9
:109D5000FFF76EFF18B19DF90430002BF5DB02B060
:109D600010BD082200212046FFF762FFF7E701A996
:109D7000FFF712FF0028F2D0019AF3E70422F1E77F
:109D80000020ECE710B543681A787AB103F10C02B1
:109D900042601A7B62B90168C368C0E901128C781D
:109DA0002344036191F903100B444361104620E002
:109DB00059781A7901F03004302C1BD15C7B04F007
:109DC0003004302C1ED199780269521A02610022A7
:109DD000597811F0300F02BF816801318160997BA1
:109DE000114402690A44026193F90F301A44426136
:109DF000012010BD01F0F004202C03D1597911FB92
:109E000002F2E5E701F0C001802908BF0422DFE784
:109E100009B9034B1970034B1B6803B1184770470E
:109E20006C4A0020A04A00201F4B204A1B6800BF3C
:109E300000BF00BF00BF00BF00BF00BF00BF934214
:109E40002FD000BF00BF00BF00BF00BF00BF00BFDA
:109E500000BF00BF00BF00BF00BF00BF00BF00BF0A
:109E600000BF00BF00BF00BF00BF00BF00BF00BFFA
:109E700000BF00BF00BF00BF00BF00BF00BF00BFEA
:109E800000BF00BF00BF00BF00BF00BF00BF00BFDA
:109E900000BF00BF00BF00BF00BF00BF00BF00BFCA
:109EA00000BF0138C3D17047284700200024F400C8
:109EB00018DF70471FB50023CDE9013303936846CF
:109EC00002230093FFF7F4FF05B05DF804FB0000E8
:109ED000074A136829B923F00303136043682BB1C1
:109EE000184723F0010343F00203F6E7704700BF71
:109EF000204F0020F0B50346186880F308885868A2
:109F0000FF2464B2EFF30585002D01D1A64600477A
:109F10002546064621273FBAF0B400240025002636
:109F20000027F0B4F92040B2004700BFF0BD00BFE9
:109F300013DF7047074A4FF0FF3108B5C2F88010B1
:109F40000346FFF7F5FF20B91846BDE80840FFF7C4
:109F5000D1BF08BD00E100E0024A1368013B136075
:109F6000704700BF244F0020704768DF704767DFED
:109F7000704763DF7047ADDF7047A9DF7047A8DF28
:109F80007047A6DF704700007FB50023CDF80A3088
:109F9000ADF80E3001238DF80A300DF10603ADF84F
:109FA0000810049302A9044BADF806200593FFF7AF
:109FB000E8FF07B05DF804FB284F002010B40D4BFC
:109FC000024618884FF6FF7398420FD00A4B1B6861
:109FD000DB070BD5094B60245A7099701C70084B35
:109FE0005DF8044B99890322FFF7CEBF08205DF886
:109FF000044B70472E4700201C4F0020284F0020A4
:10A00000F24E002010B4154B024618884FF6FF732D
:10A0100098421FD0124B1B68DB071BD5114B6024E5
:10A020001C7003245C7001249C70140ADA701C718B
:10A03000140C120E9A710A0AD9711A720A0C090EBE
:10A040005A7299725C71084B5DF8044B99890B2226
:10A05000FFF79ABF08205DF8044B70472E47002099
:10A060001C4F0020284F0020F24E0020A5DF704733
:10A07000A2DF7047A0DF704786DF70477FDF704741
:10A080007DDF70477CDF70477ADF704776DF70478F
:10A0900074DF704773DF704772DF70476DDF7047A2
:10A0A0006CDF7047704761DF704760DF704710DF1B
:10A0B000704748DF704700002DE9F743224E234FD9
:10A0C00033683A68B3FA83F56D09002A37D0DFF8B0
:10A0D000808098F8003003F0FF044BBB01A8FFF725
:10A0E000E8FF05281FD010B93B6801989847E5B9EB
:10A0F000174DDFF86080DFF860902B78C3B9B8F8AF
:10A100000030ADF80430D9F8003001A91846FFF747
:10A11000CAFF05280FD010B9326818469047002CA6
:10A12000EBD12546D3E70124E1E70125002CD0D06F
:10A1300003B0BDE8F083002CFAD10124F1E7002B35
:10A14000F6D00124D4E700BF9C4A0020FC4F002039
:10A15000F84F0020984A002014500020024B1B7832
:10A160000BB1FFF7A9BF7047F74F00200C4B1B78CE
:10A17000062B10D10B4B1B681A070CD10A4B186821
:10A1800000F0F003302B08D000F0E000A0F1400315
:10A19000584258417047002070470120704700BF67
:10A1A000E00F00F0E40F00F0E80F00F0094B1B781F
:10A1B000062B0CD1084B1B681A0708D1074B1868EF
:10A1C00000F0F000A0F130035842584170470020E1
:10A1D000704700BFE00F00F0E40F00F0E80F00F060
:10A1E000BFF34F8F0549064BCA6802F4E062134380
:10A1F000CB60BFF34F8F00BFFDE700BF00ED00E075
:10A200000400FA05084B5A6E013A5A6622B907490A
:10A210000A7822F002020A701A6E0132042A08BF7C
:10A2200000221A66704700BF4C4F0020184F0020D4
:10A2300028DF704729DF7047D0E9003018477BDFFF
:10A24000704775DF7047000037B5164B18884FF61A
:10A25000FF73984210D0144A144D1378297B0133B0
:10A26000DBB2994213702C4608D31149FFF7E9FF7E
:10A2700010B1AB6903B1984703B030BD0023137030
:10A280002B7C33B13B21FFF701FF10B1AB6903B168
:10A2900098476369002BEFD000228DF8042001A8B5
:10A2A000E9E700BFA64A002010500020A84A00207D
:10A2B000444F002030B53AB11368DB430A4D0144E6
:10A2C000884204D1D84330BD4FF0FF33F6E710F891
:10A2D000012B5340082213F0010418BF2C46013A09
:10A2E00084EA5303F7D1EBE72083B8ED10B5084BB0
:10A2F0009A685AB150B9EFF3108172B6054A1C68DA
:10A3000014605C685460986001B962B6002010BDAA
:10A310001C50002000E100E010B50A494A788C7812
:10A32000531CDBB29C4208BF00230C789C421FBF29
:10A330000370486802EB420200EBC20008BF002035
:10A3400010BD00BF384F002073B5154E736823B39E
:10A35000144D6B690BB300240DF107002C748DF8BC
:10A360000740FEF74DF90DF10600FFF7D5FF90B15C
:10A37000022303709DF80630456073709DF8070056
:10A38000FFF7B4FF24B9084B4FF48012C3F8002143
:10A39000204602B070BD0424F0E70824F8E700BFAF
:10A3A000384F0020C44A002000E100E02DE9F347C7
:10A3B000334B344A5B881188334DDFF8E080994293
:10A3C0000BD852889A4208D36B69002B56D10023D0
:10A3D00088F8003002B0BDE8F08798F800403CB142
:10A3E0006B69002BF3D000228DF8042001A841E016
:10A3F000264ADFF8AC901278D5E90163002A18BF2D
:10A400001E46D9F80430002B36D0042E2DD9204F0B
:10A410007B698BB37B7C8DF80440012B01A80CBFBA
:10A42000B2464FF0000AFEF7EBF80DF10300FFF71C
:10A4300073FFC0B101230370164B4760D3F8043596
:10A44000C0E904A4C0E902369DF8033089F8013060
:10A450009DF80400FFF74AFF44B90F4B4FF48012F8
:10A46000C3F80021B3E70424F2E70724AB69002B0B
:10A47000ADD020469847AAE70824F7E70122B3E7C2
:10A48000E44A0020444F0020A84A00201050002039
:10A49000C44A00200010014000E100E0A44A00206E
:10A4A000384F00200C4B0D484FF4003210B5C3F864
:10A4B000802001244FF48033C0F84833C0F80833BB
:10A4C0004460FEF757F8064B846000201860FEF7E2
:10A4D00051F8044B187010BD00E100E0001001407D
:10A4E0000C500020F64F0020F8B5124C124D2646B5
:10A4F00022782B789A4200D1F8BD23780F48104A71
:10A50000078812680F48DBB219B202EBC10C006871
:10A5100052F83120BCF8041003FB070090470A4AA8
:10A5200023781288DBB29A4286BF0133DBB2002364
:10A530003370DDE7C44F0020B44F0020C04F00202F
:10A54000BC4F0020B84F0020C24F002038B5064C49
:10A55000064D636E042B00D038BD2846FFF764FC1F
:10A56000FFF7C2FFF5E700BF4C4F0020A0860100B7
:10A570005B689A68054B9A4206D1D0E901230449E9
:10A580000132013B0A604B60704700BFACCD070051
:10A59000904A002008B5084E084CA41BE40800258A
:10A5A0000436AC4203D056F83530984708B1FFF76F
:10A5B00017FE0135F5E700BF48470020504700204F
:10A5C0004FF0A043D3F81005C0F3807070474FF0F0
:10A5D000A0434FF4805241B938B9C3F808254FF071
:10A5E000A0430322C3F830277047C3F80C25F6E7D1
:10A5F00070B543F208031C68164B1968A1F5405169
:10A60000091B814224D3144B144E1D6A3460012D62
:10A610001AD19A6902F6FF7222F47F6222F00F02C9
:10A62000891A88424FF0000103D9C3E90451183355
:10A6300004E02244C3E90415326024330022C3E954
:10A6400001221860104670BD0022C3E90422EEE723
:10A650000420F8E71410001054510020144F00207B
:10A6600070B59CB00023002210930023CDE9122383
:10A670004C4B4D4A4D4C4E4DCDE914234D4BCDE93D
:10A6800016434D4BCDE918534C4B1A9303F17453B9
:10A69000A3F52303A3F692431B9309B1002852D0DC
:10A6A000044645180026A54250D1454D2C68002C83
:10A6B00049D0109A1CA9531C372A0A444FF0800134
:10A6C00002F8701C4FF0000260D8382B57D1DDE93A
:10A6D000122310980821E1FB00231046194612BAF4
:10A6E000CDE912010F9269461A0A8DF83B308DF8B8
:10A6F0003A2008461A0C1B0E8DF839208DF8383098
:10A70000FDF7A4FF621E00231B99D94002F8011F28
:10A710001A99D94011711999D94011721899D940D3
:10A7200011731799D94011741699D940117515995B
:10A73000D94011761499D9400833202B1177E3D1F1
:10A740006B60002000E00E201CB070BD109B14F860
:10A75000011B1CAA1A440133402B02F8701C1093F1
:10A76000A1D169466846FDF771FF129B139A1096B6
:10A7700013F5007342F10002CDE9123293E70DF8B0
:10A7800003200133A1E70DF8032001333F2BFAD951
:10A7900069466846FDF75AFF382200216846FDF7F2
:10A7A000C1FE94E785AE67BB67E6096A72F36E3C4B
:10A7B0007F520E513AF54FA58C68059BABD9831F8C
:10A7C000904A0020044A0023036043608360C2E98A
:10A7D0000C33C2E9043370475451002010B50C49C2
:10A7E0004A6E042A044611D00B6E1344032B02F167
:10A7F00001024A6688BF043B182202FB0313184675
:10A800000021FDF78FFE2060012010BD0020FCE735
:10A810004C4F002030B5044685B00D461022002173
:10A820006846FDF77FFE237A012B0AD0022B0ED05B
:10A8300063680193236829469B686846984705B07A
:10A8400030BD23690293A38AADF80C30F0E70123F1
:10A85000A2898DF80030E389ADF80A20D31AADF84B
:10A860000830E5E738B51C4B5A6E19465AB31C6ED2
:10A87000182202FB04331A7A012A07D0022A23D0B5
:10A8800018460921BDE83840FFF7C4BF1825D88A0B
:10A890009A8A05FB0414D4E90314121AB2F5806FE6
:10A8A0004FEA80000144B4BF92B24FF4806220446A
:10A8B000FFF7C0FC11280BD1084A137823F00203DC
:10A8C00043F00403137038BD9889FFF7B1FCF1E73A
:10A8D0000028F8D0D4E700BF4C4F0020184F0020CC
:10A8E00038B52A4A13780146980742D5284A146E8B
:10A8F0001820022900FB042005D003292DD0BDE833
:10A900003840FFF7AFBF234B00211970037A012BAA
:10A910000CD0022BF3D18389028A01338381C3894E
:10A9200001339BB29A42C381E9D111E0858AC38A7F
:10A93000E91AB1F5806FB4BF89B24FF480610B445E
:10A9400018219BB201FB04229D42D382D7D1002162
:10A95000FFF760FFFFF756FCD1E70E4A137801338B
:10A96000DBB2032B01D81370C9E700231370082151
:10A97000EEE75907C3D50649496E03F0FB03137090
:10A980000029BCD043F00203EDE700BF184F0020C0
:10A990004C4F0020F44F0020054A137813F0060FA7
:10A9A00004D143F002031370FFF75CBF704700BF90
:10A9B000184F00202DE9F043494ED6F8009019F0C9
:10A9C000040F85B0054614464DD019F0020F40F033
:10A9D000818049F001033360424B1B78DB073CD593
:10A9E000414F424B9F423AD3414B9F4237D20028BE
:10A9F00037D0C0F30B0373BB3B68984204D20520E9
:10AA000029F0010333601FE08AB27B6800EB023259
:10AA10009342F4D31FFA81F8B8F1000F19D06846B9
:10AA2000FFF7DCFE98B1009BC3E90074009B022293
:10AA30002D0B1A729D81A3F81080FFF7ADFF3368CC
:10AA400043F001033360002005B0BDE8F083072028
:10AA5000D6E70420D4E70620D2E70120D0E7022081
:10AA6000CEE70320CCE7C0F30B03ABBB214E0F4670
:10AA70004FF0020C3246C6F804C5D2F800E4BEF12D
:10AA8000000FFAD0C2F80805D2F800E4BEF1000FBA
:10AA9000FAD0C2F80435D6F800E4BEF1000FFAD0BF
:10AAA000013F00F58050E6D105EB0136B4B13946DF
:10AAB00010226846FDF736FD310B01232D0BADF852
:10AAC0000A10684639468DF800300194ADF80850F8
:10AAD000A047B8E70A20B7E70620B5E72046B3E766
:10AAE000204F0020184F0020384700203847002012
:10AAF0004847002000E001402DE9F0430F46464959
:10AB00001C460B6813F0040F85B00546884646D0F6
:10AB10009E0777D443F001030B60404B1B78D807A6
:10AB200072D53F4E3F4B9E4270D33F4B9E426DD2FB
:10AB30001FB9032005B0BDE8F083002DF9D047EA26
:10AB40000503990701D00620F4E733689D425FD3DF
:10AB500093B2716805EB8303994259D31FFA82F9C6
:10AB6000B9F1000F01D10420E4E76846FFF736FE93
:10AB700098B1009BC3E90064009B01221A72C3E9EB
:10AB80000375A3F81490FFF707FFD8F8003043F0DF
:10AB90000103C8F800300020CCE70720CAE7002FE7
:10ABA000C7D00028C5D047EA00039B07CBD1002AB5
:10ABB000D9D01E4B0121C3F80415D3F80014002985
:10ABC000FBD01A490023084657F8236045F8236054
:10ABD000D1F80064002EFBD001339A42F4D1002357
:10ABE000C1F80435D0F80034002BFBD000268CB11E
:10ABF000314668468DF80060CDE90145ADF80C207E
:10AC0000A047C8E70A2095E7012093E7022091E7D3
:10AC100005208FE720468DE7204F0020184F0020A9
:10AC200038470020384700204847002000E0014016
:10AC3000F8B51E4C1E4F0646254623789BB90123C6
:10AC400023701C4B1C4C1E60FFF780FC002201216E
:10AC50002046FFF7AFFE07280246F5D048B1002393
:10AC60002B700320F8BD3846FFF7DEF8FFF73CFCF9
:10AC7000E3E7124C124F134E5821201DFFF71AFB29
:10AC8000214620604FF4AE720E480B4C01F0D2FF0B
:10AC9000FFF75CFC3B46572231462046FFF72CFF6E
:10ACA0000728F5D00028DDD0D9E700BF6C4A002086
:10ACB000A0860100A04A002000F0070054510020A7
:10ACC000119E0700005300202DE9F04F1E4E1F4932
:10ACD000726B336B02F6FF74E41A0C40A50805F69C
:10ACE000FF7585B003F580570D4003EB00080AB1EE
:10ACF000934226D04FEA95094FF0010A4FF0030B1B
:10AD00006846CDE900A8CDE90279FFF7D1F8A8B9E6
:10AD10006846CDE900B7CDE90289FFF7C9F868B9FF
:10AD2000A542736B8CBF0446641B1B1B00202F4481
:10AD3000A8443363FFF77CFF002CE1D105B0BDE8E8
:10AD4000F08F0020FAE700BF5451002000F0FFFF11
:10AD50007FB5124B0C685B6B1D18E41A032300933C
:10AD60000F4BA4086846CDE901350394FFF7A0F81E
:10AD7000064638B90846FFF725FD3046FFF758FF6D
:10AD800004B070BD102200216846FDF7CBFB684679
:10AD9000CDE90154FFF78CF8F2E700BF54510020D1
:10ADA0000080070030B54268527802F00F01082990
:10ADB00087B003460FD103691C6800250CB907B0A2
:10ADC00030BD214625736846FEF7F4FD6846FFF75F
:10ADD000E9FFA468F2E712F0C00120D102F03000D0
:10ADE00010280ED15A6911705A68186953789468FE
:10ADF00003F00F03072B09D10146204600F017F896
:10AE0000DDE79006F0D55B691970D8E71279214625
:10AE100014B101F00FFFD2E7FDF784FBCFE78029E3
:10AE2000CDD10069002192060160C8D5EBE77FB55E
:10AE30000023CDE902318378194490F9033004915D
:10AE4000194403780591CDE900003BB16846FFF74E
:10AE5000A9FF6846FEF796FF0028F7D107B05DF816
:10AE600004FB00002DE9F04355686B7813F0C00433
:10AE700089B006468C46174603D0402C6AD0002481
:10AE80000AE003F00F025E4903F03003102B51F883
:10AE9000228020D004D8CBB1204609B0BDE8F08391
:10AEA000202B1ED0302BF7D17B6929781970072A07
:10AEB0000AD17B6838691A792146FDF733FB7B6834
:10AEC00039699868FFF7B3FF3A6940E03A69294663
:10AED000C0470446E0E77B6901221A703A69796845
:10AEE000F6E7BCF1020FD7F8149024D1042A22D837
:10AEF00004A9FEF784FE04460028C0D0069B2BB1AF
:10AF0000796899F800304A799A4205D8059B7360B0
:10AF1000069B002BC0D0B2E708793A6900FB0322F8
:10AF200004A8C04728B199F80030013389F80030EF
:10AF3000E4E70446EAE799F800306A799A429ED934
:10AF40003A692979581C89F8000001FB03227968C5
:10AF50003046BDE7D2F81080454655F8043B13B99A
:10AF6000FEF7EAFEB5E7022914D104A9FEF747FE71
:10AF7000002884D0D8F8003079682A4604A8984779
:10AF8000044600283FF47BAF069B002BF2D1059BC3
:10AF9000736081E701292BD04CB24CB105297FF4B5
:10AFA0006EAF04220DEB0201FEF742FE042424E002
:10AFB0000DF1040901340B2C3FF461AF0122494625
:10AFC0003046FEF735FE00283FF459AF19F9013B32
:10AFD000002BEFDB0B4B049301ABCDE905340023D1
:10AFE0000793D8F8003079682A4604A8984770E794
:10AFF000082201A9FEF71CFE08240028EAD13EE73A
:10B000007CCC0700EF9907002DE9F04F8B788FB0CB
:10B010000025CDE904521A4491F903300692CDE996
:10B020000055CDE902111A44044607924FF0010879
:10B03000A3682BBBDDE9033402A85D78FEF7A2FE0E
:10B040000028F7D115F0300F03D1039B1B7803B113
:10B050000134002C65D06309002293425BD10EAA13
:10B0600002EB830304F01F044FF0FF30C4F120040F
:10B0700020FA04F453F8380C231A5842584108E0D7
:10B0800008A92046FEF788FD30B9A368002BD1D06F
:10B0900000200FB0BDE8F08F089EDDF80CA0002E58
:10B0A000C8D0F70806F00706039B1A78974204D128
:10B0B0005B7803F00F02082A58D102A8FEF762FE5F
:10B0C000DDF80C90CA45EFD1BD420DD8039A5378F4
:10B0D00003F00F03082B29D002A8FEF753FE039BB1
:10B0E0009945F3D14FF0FF3531462046FEF724FE57
:10B0F00000289DD1CCE79B681B789F4233D14946FD
:10B1000008A8FEF757FC89F80C8008AA31462046AB
:10B11000FFF7A8FE25E05DF822100131B8D1013219
:10B120009BE70120B5E79A45DED081E71578BD425F
:10B13000DAD8069BD4F808A0D3F80090A368B9F138
:10B14000000FF0D09A457FF473AFD9F80030D3F8F0
:10B1500000B0BBF1000FCED033463A4649462046F8
:10B16000D847002894D0D9F80890E7E713F0300FBB
:10B170000FD1049B3F2B0CD85A090EA901EB820278
:10B1800003F01F0352F8381C08FA03F30B4342F88C
:10B19000383CD4F80C90B9F1000F04D002AB324621
:10B1A00039462046C84702AA31462046FFF75AFED4
:10B1B0009EE7F0B585B00E468C6869460746154691
:10B1C000FEF71DFD88B1B06878B1737803F03003E5
:10B1D000202B03D129462046FFF729FE2A46214687
:10B1E0006846FFF711FF019B7B6005B0F0BD0000D2
:10B1F00070B50D4B0D4C9A6B0D4E0E4D0E492160E6
:10B200005C33C4E901320D4BE3600D4B0022314643
:10B210002846C3E90022FFF70AFE324629462046A7
:10B22000FFF7F2FE70BD00BF54510020F052002025
:10B230002850002028CE0700EF99070071A50700CD
:10B24000904A00202DE9F341002406460DF1070045
:10B250000D4617468DF80740FDF7D2F9204B214ADD
:10B2600018781178CBB2204909888B4238BF013356
:10B27000C0B238BFDCB2A04228D014781378DBB259
:10B28000994286BF0133DBB2002313709DF807009B
:10B29000FFF72CF84FF6FF739C421ED0134B1B6830
:10B2A00003EBC40843F834709EB195B1104B188875
:10B2B000104B1B682A46314604FB003001F0BAFCF3
:10B2C000A8F80450002002B0BDE8F0814FF6FF74EA
:10B2D000DCE70020A8F80400F5E70420F3E700BF4E
:10B2E000C44F0020B44F0020C24F0020BC4F0020AC
:10B2F000C04F0020B84F002007B5084B1B88072B14
:10B30000CDE9000107D9064A08216846FFF79AFFF0
:10B3100003B05DF804FB0920FAE700BFC04F00202E
:10B3200039A207000021024A0846FFF78BBF00BF81
:10B330005DA1070070B52A4E356815F002018AB08C
:10B340004CD1102201A8FDF7EDF80B23ADF8023027
:10B35000244B059345F60213ADF818300DF10201A8
:10B36000FE230DF11D008DF81A30FEF789FE04460C
:10B3700048BBBDF802100B2928D84B1C8DF81B3098
:10B38000092319448DF81C3089B200231A46C9B22A
:10B3900005A8FEF781FE0446A8B98DF804000290C6
:10B3A0008DF80C002823ADF8100001A8ADF80E3080
:10B3B000FEF770FE044630B9014645F00205012053
:10B3C000FFF705F9356020460AB070BD0C238DF8F3
:10B3D0001B3008238DF81C301421D6E70024F2E737
:10B3E0001C4F0020020106032DE9F04194B04FF4F8
:10B3F00004330493FEF75EFD0446002840F03F81CD
:10B40000B048FEF795FD0446002840F03881AE4B69
:10B41000AE4A1A60AE4B4FF498721A80AD4BAE4AEA
:10B420001A60AE4A1368C3F340331BB14FF40051A6
:10B43000C2F88010AA4904A8FEF739FE002800F0DF
:10B4400022811BB1A54B4FF400521A601622002135
:10B450000DF13600FDF766F80022139240F201125A
:10B46000ADF83C20F722ADF844209E4A019201231A
:10B47000019A089208A90DA8ADF834308DF83E3035
:10B48000FEF713FE019A0446002840F0F880FB22E4
:10B4900008A926208DF82020FEF767FD9DF82020C2
:10B4A00008A942F0010203208DF82020FEF75DFD7F
:10B4B0008D4A8E49116008A81122CDE90D448DF8FE
:10B4C0001020FEF7EBFD0446002840F0D8809DF8E0
:10B4D000212008A801328DF82120FEF7E1FD044665
:10B4E000002840F0CC800722814904A8FEF7CAFD5D
:10B4F0000446002840F0C3807E494FF0C8720DA872
:10B50000CDE90D12FEF7C0FD0446002840F0B780DB
:10B51000794A8DF80A304FF6FF7111804FF6596263
:10B52000ADF8082002A9754A1846FEF7A3FD0446A7
:10B53000002840F0A480724B04AC03F11005186899
:10B540005968224603C20833AB421446F7D16B4D0B
:10B5500004A8A91CFEF70DFD0446002840F08F80CA
:10B5600001461C220DA8FCF7DDFF9DF83430ADF834
:10B57000004043F004038DF83430AB788DF80E3082
:10B580000223ADF80C301423CDE90A44ADF82C3079
:10B590002B460C94274604F0F80444F003044FF0C3
:10B5A000110803AE08AA0DA933F8040B8DF8024068
:10B5B0008DF801800896CDF824D0FEF759FD044699
:10B5C00000285CD101461C220DA8FCF7ABFF9DF8BA
:10B5D0003430ADF8004023F0180343F018038DF821
:10B5E0003430AB788DF80E300123ADF80C3007F015
:10B5F000E80343F013038DF802301723CDE90A4422
:10B60000ADF82C302B4608AA0DA933F80C0B0C947E
:10B610008DF801800896CDF824D0FEF729FD044668
:10B6200068BB384A384D136843F001031360014684
:10B6300018220DA8FCF776FF40F6CD424FF4804368
:10B64000CDE90E2303238DF84030304B13930DAC1E
:10B650000FCC0FC594E807002D4B85E807002D4857
:10B660001F70FEF7ECFD044648B92B4B4FF6FF72F6
:10B670001A802A4B1F702A4B5B68C3B908242046E6
:10B6800014B0BDE8F081274B01221A70134A92F8DA
:10B69000163358067FF5DAAE234B996819B11A684C
:10B6A00042F48002D1E64FF480031360CEE61F4BD4
:10B6B0001A7C002AE2D11E4A5F745A61FFF73AFEF3
:10B6C0000446DCE7008007001450002034490020C5
:10B6D000984A00200C4F002025B3070000E100E04D
:10B6E000A5A00700C84600209C4A002089B7070093
:10B6F000A0CC07000C0018002E470020F24E0020BE
:10B700006CCC07001C4F0020A84A0020699F07004E
:10B71000A44A0020444F0020A64A002010500020D8
:10B72000384F0020F74F00201C500020C44A002052
:10B7300049A2070010B5114C21684A071BD441F0FB
:10B7400004030F482360FEF76FFB0E4B18884FF67B
:10B75000FF73984204D01321FEF798FC48B110BD46
:10B760008B0706D5FEF794FC0028F8D141F00601BE
:10B770002160FEF7E9FD0020F1E700BF1C4F00202B
:10B78000C0D401002E4700202DE9F04F0388112B73
:10B790008DB0044639D010D8102B23D02388142B19
:10B7A00000F08D8355D8102B00F0AE8045D8022BC9
:10B7B00000F0BE800DB0BDE8F08F122B36D0502BBC
:10B7C000ECD1A54DC288EB899A42E7D1038A022BBE
:10B7D000E4D1837CD90715D4FEF7B6FD0028DDD06F
:10B7E000AB691FE09D4B82881A8000F1100303CBE8
:10B7F0009B4A9C4B1060516000221A70964BDB896B
:10B80000002BCBD1FEF7D2FDC8E7944B4FF6FF7269
:10B810001A80944B00221A70FEF796FD0028BDD0C6
:10B820008D4B9B69002BB9D09847B7E700F108030F
:10B8300003CB8B4A10605160E4E7112B71D0132BBE
:10B84000B8D1894800231A4685210088FEF716FCE6
:10B85000B0E7522B00F03A8346D8502B00F03D83DE
:10B86000512BA7D1A579002DA4D01022002108A822
:10B87000FCF758FE022D9DD17C4E2289B3899A4255
:10B8800098D1A37B043B022B94D99DF82630318AB2
:10B8900043F001038DF82630238AADF82830638AFF
:10B8A000ADF82A3004F114030B930023ADF81A30DD
:10B8B00005AB07936C4B1D8802228DF82020ADF854
:10B8C0001820284606AAFEF7D1FB002836D19DF89D
:10B8D0001430DA0732D440F2FD1308A92846ADF837
:10B8E0002430FEF74CFB65E7552B00F01884562BEF
:10B8F0007FF460AFA379002B7FF45CAF5A4B132128
:10B900001888FEF7C3FB55E701210020FEF75FFE14
:10B91000554BA2881A80564A136823F0020313601D
:10B9200048E7FFF707FD504B4FF6FF721A8041E7DB
:10B930004D4B00211888FEF71AFB3BE7002308A9AE
:10B940002846ADF82430FEF71AFB00287FF432AF0A
:10B95000CDE908000A90207D431E052B00F2AD8240
:10B96000DFE813F00600340244029E00AB025A02E4
:10B97000638A062B01D0032116E03E4BD4F8165003
:10B980001A883D4B0A951A80637D099301229342E0
:10B990008DF820200CD1394A1370384B1C78012CBB
:10B9A0000AD0022C1BD005210120FEF707FB01E77E
:10B9B000022BF0D00721F7E7002DDCD0B5F5807F12
:10B9C00045D82F4E2F4B00271C22394606F13C004C
:10B9D0001F70FCF7A7FD3763B5630121E4E7002D75
:10B9E000C9D0C5F30B0333B1254B274A5B6D1268F1
:10B9F0002B449342BFD1B5F5805F28D8214B1B78EB
:10BA00003BB31F4B204A586D12682918914220D829
:10BA1000DA6C1865C3E911521C4A186313781C4C80
:10BA2000013303F0030313701A4B00221A802368BA
:10BA3000194A01332360194B1B6801211844FEF792
:10BA4000B9FF0028C9D02368013B2360ABE704217C
:10BA5000AAE70821A8E700BFA84A0020A64A0020BC
:10BA6000E44A0020105000202E470020F24E002013
:10BA70001C4F0020404F0020424F00202C47002048
:10BA80005451002011500020104F0020EC4A00209B
:10BA9000244F0020F04E0020599F0700144F002033
:10BAA00003238DF82030974B1C78012C04D0022CF6
:10BAB00000F0D6800524ADE0934FD7E90E219142E6
:10BAC00040F08281914E3378002B40F0A380FFF745
:10BAD0008FFB0128EED18E4B93F874201C46002A70
:10BAE00000F0B98093F87A30002BE3D0894DD5E986
:10BAF0000001A8B1A1B194F8DB3013B194F8DC30A7
:10BB000073B994F884305BB1D4F88830342B07D102
:10BB100094F88CC0804A002343F20C0E634501DB8D
:10BB20000A2477E052F8049BBEF80080C14500F07B
:10BB3000FC820133F2E794F87C30002BF0D0BA6835
:10BB4000D4F880309A42EBD894F8E830002BE7D153
:10BB5000724B2B6020236B60FEF782FD0028DFD143
:10BB600094F8E9706E4B6F493A46184601F062F856
:10BB70006D4A402F0346C2E900079BD1296800297E
:10BB800098D011F0030795D1684A00926A68684816
:10BB9000FDF760FC00288DD0664D94F8A1302F6031
:10BBA000032BBDD8DFE803F00C39294194F87C3031
:10BBB000002BB5D0FA68D4F880309A42C4D3AFE7EE
:10BBC00094F8B030002BABD0D4F8B4302B605A4B83
:10BBD000524C03F1200718685968224603C2083303
:10BBE000BB421446F7D1286880B3FEF701FD80B947
:10BBF0000124FFF71DF834700CE094F8A830002BF6
:10BC00008ED0D4F8AC202A604C4BC3F5FC239A426A
:10BC1000DDD9042421460420C7E694F8A230002B85
:10BC20003FF47EAFD4F8A430D0E794F8A830002BCE
:10BC30003FF476AF94F8A230002B3FF471AFD4F804
:10BC4000A430D4F8AC20991829600BB90324E1E79B
:10BC5000002AD9D1FAE71B78002B7FF461AF29E7DE
:10BC6000294CD4E91423616CD31A9942264640F03A
:10BC7000AB80A36C62650020E3646064FEF7D8FFCC
:10BC80002C4B216D1A689142984632D12C4C236876
:10BC9000002B30D11E4D95F8B930032B2ED11D4FFE
:10BCA0001E4B3B60274BD8F8001018684FF0200956
:10BCB000C7F80490FEF7D4FC4A46002805F1BB0102
:10BCC000386814BF0A24012400F0A6FF002818BF1A
:10BCD00005247369A3B1012B7FF422AF1A4B012C09
:10BCE0006ED195F8A120032A68D8DFE802F031551B
:10BCF0005B6101248EE7FEF7F7FBC8E70A24E8E75B
:10BD0000124BECE72C47002054510020115000202A
:10BD100028500020904A0020B8500020704A00208F
:10BD2000B052002012510020644A0020A8CC070025
:10BD300094CF0700104F0020E35000200080070040
:10BD4000244F0020144F0020785100206C51002017
:10BD500001229A60D5F88020B260B26C5A60D8F89F
:10BD600000201A6000212022B248B34DFCF7DAFB14
:10BD7000B222FF21B148FCF7D5FB00233363B04E5C
:10BD80002846FEF755FF11287FF444AF3046FEF7F2
:10BD90004BF8FEF7A9FBF3E7A5229A60D5F8A4209B
:10BDA0007263DAE7AA229A60D5F88020F260D4E7BD
:10BDB000AC229A60D5F8A4207263F5E70A24CCE798
:10BDC0000022C3E90122CCE7082423E7638A032B7E
:10BDD00002D003210220E8E5A27D637D43EA02232D
:10BDE000984A1380984A01211380F3E704238DF8C1
:10BDF0002030964B1B78012B04D0022B08D0052154
:10BE00000320D2E5924BD3E90F01FEF7FBF8D1E412
:10BE10008F4B186D996CF8E7638A022B02D00321CF
:10BE20000620C2E5637D09930622012B8DF82020B0
:10BE300009D1864A1370854B1B78012B07D0022B42
:10BE400035D00521ECE7022BF3D00721E8E7804B42
:10BE5000D3E90F124FF480704FF6FF739D423FF409
:10BE6000A9AC7C4B1B68DB077FF5A4AC7A4B000ABE
:10BE700060241871080A1C70D97106241872080C05
:10BE8000090E5C7099720124110A9C70DA72002408
:10BE90001973110C120E587259739A73DC705C711D
:10BEA0009C710F22B1892846FEF76EF882E4684B38
:10BEB0004FF480509A6C196DCEE7032175E500238D
:10BEC0001A461946A088FEF7D7F873E400231A46ED
:10BED0001946A088FEF751F86CE4604BE2889B8815
:10BEE0009A427FF467AC0223002508958DF8203034
:10BEF000564B268A1B780A9604F11207012B0997E4
:10BF000015D0022B32D0AA464E4B1E88002E3FF48D
:10BF100051AC4D4C2388013B9BB22380002B7FF416
:10BF200049AC29465046FEF76DF8268042E4484C5D
:10BF3000D4F83CA0A36B06EB0A029A4201D9256C07
:10BF4000E2E70AF15C0032463946204400F072FE16
:10BF5000E06B04F1400206EB000A31463846C4F8B3
:10BF60003CA0FEF7A7F905462064CDE73C4B384CD2
:10BF70001B78D4F850A0A56C002BC5D0B6F5807FF7
:10BF8000C2D8636D626C06EB0A09A9EB0303934206
:10BF9000BAD804F1480231463846FEF78BF93149E8
:10BFA000DFF8C8A00B78BAF80020A0644FEA032B92
:10BFB0002D4BC4F8509005460BEB02001844B31803
:10BFC000FF2B0393884659D83246394600F032FE9B
:10BFD000039BAAF80030CA46244E3288002A93D028
:10BFE000636D206B616CD31A03448B428CD3204B5E
:10BFF000204FD3F800C03B6898F800E01A4901339D
:10C0000003323B6092081C4B01EB0E216044FEF7AB
:10C0100073FD002879D1236B32881344236398F889
:10C020000030013303F0030388F80030002333802D
:10C030006AE700BF8C51002095A50700B051002091
:10C04000A0860100404F0020424F00202C470020D6
:10C05000545100201C4F0020284F0020F24E002099
:10C0600011500020EC4A0020F04A0020F04E002041
:10C07000144F0020244F0020599F0700C2F5807301
:10C080009BB21A463946039300F0D4FD039B206B04
:10C090002E49F61A1F440A962D4B2E4E09971F68FB
:10C0A00033684FF480720133AAF8002033604022D5
:10C0B000294B59443844FEF71FFDE0B9BAF8002077
:10C0C000236B13442363CA4698F80030234F0A9E1B
:10C0D000013303F00303002288F800303A80002E79
:10C0E0003FF47AAF19480999324600EB032000F07B
:10C0F000A1FD3E8070E73368E56CD4F854A0A564D8
:10C10000013B3360C4F850A0DEE73B68E56CD4F82F
:10C1100054A0A564013B3B60C4F850A07FE7F72121
:10C12000A088FDF728FFFFF745BB94F8A120032A5C
:10C130003FF6F6AC01A353F822F000BF37BB07006F
:10C1400049BB0700ADBB0700ADBB0700F04A0020AC
:10C15000144F0020244F0020599F0700F04E00206C
:10C16000044B1B6803B11847034B1B780BB1FDF759
:10C17000A3BF70470C4F0020F74F002008B5FEF713
:10C1800015F810B1774B784A1A60FDF7EFFF28B128
:10C19000764B774A1B68C3F342331360FEF706F809
:10C1A00020B1744AD36823F08073D360FDF7DEFFBB
:10C1B00040B14FF080430022C3F80C21C3F8102196
:10C1C000C3F83825FDF7F2FF10B16B4B03221A605C
:10C1D000FDF7ECFF40B1694B05221A6001229A6716
:10C1E00000229A603F225A60654B1B78062B50D183
:10C1F000644B1B6819074CD1634B1B6803F0F003B9
:10C20000502B46D14FF08052604BD2F80414C3F843
:10C210002015D2F80814C3F82415D2F80C14C3F86A
:10C220002815D2F81014C3F82C15D2F81414C3F83A
:10C230003015D2F81814C3F83415D2F81C14C3F80A
:10C240004015D2F82014C3F84415D2F82414C3F8CA
:10C250004815D2F82814C3F84C15D2F82C14C3F89A
:10C260005015D2F83014C3F85415D2F83414C3F86A
:10C270006015D2F83814C3F86415D2F83C14C3F82A
:10C280006815D2F84014C3F86C15D2F84424C3F8EA
:10C290007025FDF76BFF28B13D4B3E4A1B6803F04C
:10C2A0004F0313603C4AD2F8883043F47003C2F85D
:10C2B0008830BFF34F8FBFF36F8F4FF01023D3F849
:10C2C0000C22D2071ED5354B0122C3F80425D3F822
:10C2D0000024002AFBD04FF01022D2F80C3223F0B9
:10C2E0000103C2F80C322D4B1A46D3F80014002972
:10C2F000FBD00021C3F80415D2F80034002BFBD08A
:10C30000FDF76EFFD3F80022002A03DBD3F80432D6
:10C31000002B23DA214B0122C3F80425D3F8002493
:10C32000002AFBD04FF010221521C2F80012D3F8DA
:10C330000024002AFBD04FF010231522C3F804225A
:10C34000164B1A46D3F800140029FBD00021C3F87D
:10C350000415D2F80034002BFBD0D1E7104B114A62
:10C360001A6008BD74C007400DF0ADBA4402001059
:10C370003C050040F0ED00E0A005004010560040F4
:10C38000E00F00F0E40F00F0E80F00F000C0004004
:10C3900058020010E40E004000ED00E000E0014013
:10C3A000284700200090D00373B500230DF1020050
:10C3B0008DF80230FCF724F9264B1B7803F0FF04BC
:10C3C000002B41D1244B1A68002A3DD0234AD2F8D1
:10C3D0000813C90738D51C601B68214D01930DF166
:10C3E0000300019BD2F808658DF80340FCF708F9BB
:10C3F0006A6829681F2A98BF541CA142F6B26C6073
:10C4000004D1202C14BF611C0021296015499DF81E
:10C4100003008E542A6894423ABFC2F121021319D4
:10C42000A31AAA689A4238BFAB60FDF75FFF6B683A
:10C430002A681F2B94BF013300239A4201BF074A89
:10C440000123C2F8083353609DF80200FDF74EFF48
:10C4500002B070BDF74F002000D1004000D0004076
:10C46000E84F0020C54F00202DE9F04FAE49AF4AFC
:10C47000AF480B68007887B004931378984200F0B7
:10C48000AE800133DBB2022B08BF00231370127899
:10C49000A84B53F82240049B234423F07F430B60B6
:10C4A00001230193A44AA5481378D0F800C050781E
:10C4B0000390506892780592A14A02900020D1F82A
:10C4C000009092F800801946624686468246039D97
:10C4D000A94240F08780BEF1000F05D0984981F84D
:10C4E00000809149C1F80090944900B10A60019818
:10C4F0000A68002840F0C780BCEB020218BF012286
:10C50000019200268E4AD1F800A012780492864A41
:10C510004FF0000CD2F80090504661464FF0010BEE
:10C52000E646002E40F0B480039A9A4240F0CF8055
:10C5300009B1814B1A70814BBCF1000F00D018601B
:10C540001B689A4502D1019A002A42D0002B00F0C4
:10C550001881D3F800907B4C734BD4F804651868AD
:10C56000794F351A3B7825F07F4503359BB94FF459
:10C570008033C4F84433C4F80433744B4FF40032AE
:10C580004FF00108C3F880211A60C4F80080FBF75F
:10C59000F1FF87F80080A9452CBF4844401920F0DE
:10C5A0007F40C4F84005D4F804359B1B23F07F433B
:10C5B000801B033320F07F4083420AD9D4F804352E
:10C5C000C4F84035FBF7D6FF604B4FF40032C3F898
:10C5D00000215B4B00221A7007B0BDE8F08F0024E9
:10C5E00001945FE7029E01EB410506EBC5070131AF
:10C5F000059EC9B2B14208BF0021029E16F835500F
:10C60000022D0AD0032D7FF462AF002A3FF45FAF02
:10C6100082F810A00120D269F7E7D7F804B01546D8
:10C620001646002D3FF453AFAB4500F0AD802E46CB
:10C63000ED69F6E70120B4E0D2F800C0A44505D9C1
:10C6400005B10A60ACEB040414605BE7A4EB0C04D6
:10C650006044D2F80CC0C2F800E0D2F81C80BCF1F3
:10C66000000F07D0049DD661054425F07F45C2E93F
:10C67000015C164601254246002ADDD1002D3FF41B
:10C6800041AF0A603EE700252E462846AE46F3E756
:10C690003246F669D2F804802D4C9768A8EB09055C
:10C6A00025F07F45A54234D83D441560C2E901EE2E
:10C6B00082F810B0C2F81CE030B115680468A542D9
:10C6C0005AD8651B0560D0614FF0010C52E0029909
:10C6D00003EB430201EBC20401330599DBB299423B
:10C6E00008BF0023029911F83210012947D162686E
:10C6F000157C002D7FF418AFA7685760E768976036
:10C700002769D76064699461049C002CC2D055608D
:10C71000C0E7A9EB080424F07F44BC423ABF3C1BAD
:10C720001460C2F800E0C1E70C500020085000205F
:10C730000950002000500020384F002018500020E1
:10C74000F54F002000100140F64F002000E100E00E
:10C75000FEFF7F00ED1BE769A0463FB13C4627681E
:10C76000AF42F7D37F1B2760274644461560D76149
:10C77000E26102461046D4E680460446EFE7012116
:10C78000D2E6FDF78FFE24E7B5420AD1D269002A2E
:10C790007FF450AF08480127876091463846BE466F
:10C7A000B846D5F800B0ED69F561002D3FF48FAEC5
:10C7B0002E685E442E608AE6001001402DE9F843A1
:10C7C0002549264B0025C1F84051C1F84451C1F814
:10C7D0004851C1F84C51C1F80051C1F804511B68CF
:10C7E000002B31D0D1F804451D49DFF88880096855
:10C7F000641A24F07F442F461A68A2420FD8A41A64
:10C8000015441A7CDE694AB1D8F800901F74D3E948
:10C810000521B9F1000F1BD01046C847B6B9114A1F
:10C82000114B11781B788B4205D10133DBB2022BFF
:10C8300008BF0023137012780C4B43F822500C4BA6
:10C840004FF48012C3F80021BDE8F8833346D3E7E4
:10C8500008469047E2E700BF001001401850002052
:10C860000C500020095000200850002000500020EB
:10C8700000E100E0084F00202DE9F047002186B0DC
:10C880000846FDF7A4FE4FF0A0430422B04CC3F8C5
:10C890007827B04BB04900254FF4AE7220468DF892
:10C8A00007501D7000F0C6F92668721C06D02A4693
:10C8B0005821201DFDF7FEFC86420AD04FF4AE72CF
:10C8C0000021A348FBF72EFE012300206360FEF742
:10C8D000AFF943F208031E682369012B18D063697E
:10C8E000B3B1A5699D4F05F6FF7525F47F6525F069
:10C8F0000F053544BB68A52B77D00CD8012B19D078
:10C90000FDF75EFE002800F00E8140F6B8358FE09E
:10C910003546934FEEE7AA2B77D0AC2BF0D12846C3
:10C92000FEF7D2F9064600286BD139462846FEF7B5
:10C930000FFA65E06369012BE2D1276BD4F82490EC
:10C940003E444FF0030AA9EB0707B7F5805F4FF0AD
:10C9500000024FF001013046B84628BF4FF480581E
:10C96000FEF728F8034618B101238DF80730C7E712
:10C97000424629463046FEF7BFF80028F4D14FEA78
:10C98000980302A8CDE902A604950593FDF790FA55
:10C9900002460028E8D101212846FEF70BF80028BE
:10C9A000E2D1236B43442363FEF742F9B7EB080758
:10C9B00046444544C9D143F208033A4618684946FB
:10C9C000FDF778FCA36A984204BF0123C4E907037A
:10C9D000624808BFC4F81890FDF7F4FE0020FEF787
:10C9E00027F90646002EBFD18AE72846FEF76CF9E4
:10C9F000064630B93846FDF7E5FE3046FEF718F931
:10CA000006460123CDF80730ECE739462846FEF705
:10CA10009FF9E6E740F2E730FDF706FA15F0030F5D
:10CA20004FF000010CBF01200846FDF7D0FD013D8D
:10CA3000FDF7C6FD002872D0002DEBD1012108467C
:10CA4000FDF7C5FD002D6ED001238DF807309DF850
:10CA5000073013B9002D40F0C780FDF723FD414B8F
:10CA6000414A1A60414A424F424E052100259170C9
:10CA7000414915805160414A1560414A1570414A4B
:10CA80001570414A4FF48011E020C2F8801182F8FD
:10CA90001403116001F18041A1F56F21F61BC1F86B
:10CAA000085582F81103394AD1F804151160384944
:10CAB000384A0A603849A8320A60384A1570384A3C
:10CAC0001570384A08211180374A14211180F60860
:10CAD000AE4279D1354A137843F001031370344BD9
:10CAE000344A1A60344B04221A60344B00221A6014
:10CAF000A36B8BB1FEF77CFB70B1236A002B69D16D
:10CB0000A369002B66D02E4A13602D4B1868FDF7E1
:10CB10006FFD2C4B01221A70FDF7E6FCFCE7003597
:10CB200018BF01258AE7236A012B0CD8E56965B196
:10CB300043F2080300221868A169FDF7BBFB2B1A1A
:10CB40005D425D4183E7002581E701257FE700BF66
:10CB5000545100206C4A002000F00700785100205A
:10CB60006C510020084F0020F9B20700384F002018
:10CB70004847002050470020BC48002018500020A3
:10CB8000085000200950002000E100E00C50002077
:10CB9000BC4F00206C470020B84F0020B44F00204D
:10CBA000C44F0020C04F0020C24F0020184F00206B
:10CBB000FC4F0020E1A80700204F0020244F002058
:10CBC000104F00201150002057F835309847A0B979
:10CBD00001357DE7E36A002B9ED1A369002B9BD032
:10CBE0000C4B626A1A6090E743F208031A68FDF77B
:10CBF00061F910B91046FDF79DF943F208031A6870
:10CC0000FDF758F910B91046FDF794F9002006B069
:10CC1000BDE8F087104F002030B501390024A24252
:10CC200001D1002005E0035D01340D5DAB42F6D07B
:10CC3000581B30BD0A44914200F1FF3300D17047C8
:10CC400010B511F8014B03F8014F9142F9D110BD15
:10CC5000F8B500BFF8BC08BC9E467047F8B500BFE9
:10CC6000F8BC08BC9E467047C846002050EADA303F
:10CC70008883B89F604F15F30000C98E3F9B070063
:10CC8000E39A0700719A0700219D0700079D07009E
:10CC9000C99C0700899C0700B3B107000000000091
:10CCA000446675546172670008200001FFFFFFFFB2
:10CCB000FFFFFFFFFFFFFFFF00000000000000007C
:10CCC0000000000001000000FFFFFFFF512563FC92
:10CCD000C2CAB9F3849E17A7ADFAE6BCFFFFFFFFF7
:10CCE000FFFFFFFF00000000FFFFFFFF96C298D884
:10CCF0004539A1F4A033EB2D817D0377F240A46385
:10CD0000E5E6BCF847422CE1F2D1176BF551BF378D
:10CD10006840B6CBCE5E316B5733CE2B169E0F7C60
:10CD20004AEBE78E9B7F1AFEE242E34F4B60D2272D
:10CD30003E3CCE3BF6B053CCB0061D65BC86987623
:10CD400055BDEBB3E7933AAAD835C65A4F980700BA
:10CD5000F59707007D900700011101FF0100000019
:10CD600000000000021702FE64000000ACCD0700C6
:10CD7000031704FC040000004CCE07000000000074
:10CD800000000000000000000101000001000000A0
:10CD9000000000000205000021000000000000006B
:10CDA000000000000000000000000000011104FC71
:10CDB0000400000000000000021104FC0400000058
:10CDC00000000000032104FC040400000000000037
:10CDD000041101FF0100000000000000051102FE27
:10CDE0000400000000000000061104FC0400000024
:10CDF00000000000071104FC040000000000000017
:10CE0000081701FF2200000088CD0700091001FF6C
:10CE10000100000024CE0700000000000000000018
:10CE20000000000000000000011704FC700000007A
:10CE300058CD0700021704FCB400000064CE0700C0
:10CE400000000000000000000000000001010000E0
:10CE500004000000000000000000000000000000CE
:10CE600000000000010700007000000058CD07001E
:10CE700002010000010000000000000003050000A6
:10CE80004100000000000000000000000000000061
:10CE900000000000982F8A4291443771CFFBC0B543
:10CEA000A5DBB5E95BC25639F111F159A4823F9275
:10CEB000D55E1CAB98AA07D8015B8312BE853124CE
:10CEC000C37D0C55745DBE72FEB1DE80A706DC9B8F
:10CED00074F19BC1C1699BE48647BEEFC69DC10F3B
:10CEE000CCA10C246F2CE92DAA84744ADCA9B05C77
:10CEF000DA88F97652513E986DC631A8C82703B03A
:10CF0000C77F59BFF30BE0C64791A7D55163CA0647
:10CF100067292914850AB72738211B2EFC6D2C4D53
:10CF2000130D385354730A65BB0A6A762EC9C28141
:10CF3000852C7292A1E8BFA24B661AA8708B4BC2D7
:10CF4000A3516CC719E892D1240699D685350EF401
:10CF500070A06A1016C1A419086C371E4C774827B8
:10CF6000B5BCB034B30C1C394AAAD84E4FCA9C5B2E
:10CF7000F36F2E68EE828F746F63A5781478C8847F
:10CF80000802C78CFAFFBE90EB6C50A4F7A3F9BE61
:10CF9000F27871C64901B952C5EF41DE27476A559B
:10CFA00027B31CE72D1ECB0FA00C3792BE6AB2E947
:10CFB0009B2403956593690B5EF09CFDA5C02CEE48
:10CFC000F1ECA5A1470A9B3F814C5FD407D8A3147D
:08CFD00004C609D300000000B3
:08CFD80068B4FF7F01000000B6
:10CFE0000000000000000000000000000000000041
:10CFF0000000000000000000000000000000000031
:10D000000000000000000000000000000000000020
:10D010000000000000000000000000000000000010
:10D020000000000000000000000000000000000000
:10D0300000000000000000000000000000000000F0
:10D040000090D0030100FFFF258407000184070042
:10D050000010000000300800D19E07000000000012
:08D06000E9B3070035B7070032
:020000020000FC
:020000041000EA
:041014000080070051
:0410180000E00700ED
:0400000370008539CB
:00000001FF
